:020000040000FA
:100000000A128A113C2800001030A8000310A40D29
:10001000A50D0310A00DA10D031C14282308A5078E
:100020002208A4070318A50AA80B06280800103008
:10003000A800A201A3010310A60DA70D0310A00D97
:10004000A10DA20DA30D23082502031D29282208B6
:10005000240203192D28031834282508A302240894
:10006000A202031CA3032614A80B1B28080080006F
:10007000840AA80B3728080083132D3084004D30E4
:10008000A800003037208A1184288312E400F03061
:10009000831605058312E6000F306405E700670844
:1000A00066048316850008008312E4000F3083166F
:1000B00006058312E6000F306405E700670EF0398D
:1000C000E800680866048316860008002D0885008D
:1000D00008002E08860008008312EF00F0302D057E
:1000E000F1000F306F05F20072087104AD00662850
:1000F0008312E9000F302E05EB00690EF039EC0099
:100100006C086B04AE0069288312AA015F100B29EA
:10011000EF00F1019A28831203131630A0002C304F
:10012000A1000A128A11A10B91280A128A11A00BB0
:100130008F28F10A71086F02031D8B280800ED015A
:10014000EE01B92883120313F230A0000A30A10097
:100150002830A2000A128A11A20BAA280A128A11B8
:10016000A10BA8280A128A11A00BA628ED0A0319D0
:10017000EE0A6D086902A0006E086A022004031DE1
:10018000A22808008312F700770883169B001C142E
:100190001A088312F80078080800E400660883163D
:1001A0009A008312640883169B001C158B138B1313
:1001B00055309D00AA309D009C14000000008B1754
:1001C0001C119C18E1280800403083169900181172
:1001D0000800E42083168C120C12981690308312BB
:1001E000980008008312F9005F18FB280C1AF92800
:1001F000F62879089900080083128C1E02291A0833
:10020000E400042920100929981C0829181218163E
:10021000201464080800E9208A111729AE132E085B
:1002200086008316861308008316061708000E2121
:100230008A11142144308312AB00AC0107309F00B7
:100240008A113C29E900EB01690888208312EB0A36
:100250000A306B028A11031D24290800E400E6011C
:100260006408E900EA019F208312E60A0A30660268
:100270008A11031D3029080001302E2100308A1117
:10028000452000308A1154208316051283122D1642
:100290002D088500831606148611851600308A11F4
:1002A0006C2000308A11782001308312B1000130B7
:1002B000B200B401B501B601B701B801B901BA0184
:1002C000BB010A30CD000A30CE001430CF0001301F
:1002D000D0000130D1000A30D2008A15A628E900EA
:1002E0000F30E905EB0101306902031D7C29033061
:1002F000E9000130EB00BE2903306902031D8529A6
:100300000630E9000230EB00BE2902306902031D0D
:100310008E290630E9000130EB00BE290630690263
:10032000031D97290C30E9000230EB00BE29043090
:100330006902031DA0290C30E9000130EB00BE2941
:100340000C306902031DA9290930E9000230EB00D5
:10035000BE2908306902031DB2290930E9000130C5
:10036000EB00BE2909306902031DBB290330E900F7
:100370000230EB00BE290330E900EB0169080800F8
:10038000E9000F30E905EB0108306902031DCD29B2
:100390000C30E9000130EB00102A0C306902031D1B
:1003A000D6290630E9000230EB00102A0430690239
:1003B000031DDF290630E9000130EB00102A06306A
:1003C0006902031DE8290330E9000230EB00102A1E
:1003D00002306902031DF1290330E9000130EB000E
:1003E000102A03306902031DFA290930E90002309E
:1003F000EB00102A01306902031D032A0930E900CD
:100400000130EB00102A09306902031D0C2A0C3060
:10041000E9000230EB00102A0C30E9000230EB005A
:1004200069080800EF000130F1000F30EF050130DE
:100430006F02031D1E2A0330EF00512A03306F02A2
:10044000031D252A0230EF00512A02306F02031DDE
:100450002C2A0630EF00512A06306F02031D332A82
:100460000430EF00512A04306F02031D3A2A0C3089
:10047000EF00512A0C306F02031D412A0830EF00B3
:10048000512A08306F02031D482A0930EF00512A13
:10049000E9306F02031D4F2A0130EF00512A01306D
:1004A000EF006F080800EF000130F1000F30EF059A
:1004B00008306F02031D5F2A0C30EF00922A0C30C7
:1004C0006F02031D662A0430EF00922A04306F0287
:1004D000031D6D2A0630EF00922A06306F02031DBD
:1004E000742A0230EF00922A02306F02031D7B2A29
:1004F0000330EF00922A03306F02031D822A01307D
:10050000EF00922A01306F02031D892A0930EF00A3
:10051000922A09306F02031D902A0830EF00922AB8
:100520000830EF006F0808003108C0218312B100C5
:100530006B08B00031088A116C2083124D088A11B3
:10054000882083123008B4070318B50A0800310860
:100550006F218312B1006B08B00031088A116C2042
:1005600083123008B402031CB5034D088A11882891
:1005700032086F218312B2006B08B00032088A1172
:10058000782083123008B802031CB9034E088A1180
:1005900088283208C0218312B2006B08B0003208EC
:1005A0008A11782083123008B8070318B90A4E0858
:1005B0008A118828310853228312B1007108B000D3
:1005C00031088A116C2083123008B4070318B50A69
:1005D0004D088A118828310812228312B10071084F
:1005E000B00031088A116C2083123008B402031C59
:1005F000B5034D088A118828320812228312B200EE
:100600007108B00032088A11782083123008B802CD
:10061000031CB9034E088A1188283208532283121A
:10062000B2007108B00032088A11782083123008B5
:10063000B8070318B90A4E088A1188283A30F22000
:10064000E8308312A4000330A5006D08A0006E08F6
:10065000A1008A11172083122608F1002708F20052
:100660007208F40030307107F3000318F40A7308BD
:100670008A11F220E8308312A4000330A5006D082F
:10068000A0006E08A1008A11172083122208F10031
:100690002308F2006430A400A5017108A0007208CC
:1006A000A1008A11172083122608F3002708F400FE
:1006B0007408F60030307307F5000318F60A750861
:1006C0008A11F22064308312A400A5016D08A000F5
:1006D0006E08A1008A11172083122208F100230856
:1006E000F2000A30A400A5017108A0007208A10060
:1006F0008A11172083122608F3002708F4007408D3
:10070000F60030307307F5000318F60A75088A11F1
:10071000F2200A308312A400A5016D08A0006E0823
:10072000A1008A11172083122208F1002308F20089
:100730007208F40030307107F3000318F40A7308EC
:100740008A11F2202A308A11F2200D308A11F2200B
:100750000A308A11F2285230F22065308A11F220D4
:1007600063308A11F2202E308A11F22020308A1153
:10077000F22020308A11F22083126508F200303016
:100780006407F1000318F20A71088A11F2202C3074
:100790008A11F220E8308312A4000330A500690812
:1007A000A0006A08A1008A11172083122608F10010
:1007B0002708F2007208F40030307107F3000318C4
:1007C000F40A73088A11F220E8308312A40003307F
:1007D000A5006908A0006A08A1008A1117208312E9
:1007E0002208F1002308F2006430A400A50171087A
:1007F000A0007208A1008A11172083122608F300B6
:100800002708F4007408F60030307307F500031869
:10081000F60A75088A11F22064308312A400A5013B
:100820006908A0006A08A1008A1117208312220813
:10083000F1002308F2000A30A400A5017108A0000D
:100840007208A1008A11172083122608F3002708D6
:10085000F4007408F60030307307F5000318F60A48
:1008600075088A11F2200A308312A400A5016908D4
:10087000A0006A08A1008A11172083122208F10043
:100880002308F2007208F40030307107F3000318F7
:10089000F40A73088A11F2202C308A11F220E83011
:1008A0008312A4000330A5006D08A0006E08A1000B
:1008B0008A11172083122608F1002708F200720817
:1008C000F40030307107F3000318F40A73088A113A
:1008D000F220E8308312A4000330A5006D08A000C8
:1008E0006E08A1008A11172083122208F100230844
:1008F000F2006430A400A5017108A0007208A100F4
:100900008A11172083122608F3002708F4007408C0
:10091000F60030307307F5000318F60A75088A11DF
:10092000F22064308312A400A5016D08A0006E08B7
:10093000A1008A11172083122208F1002308F20077
:100940000A30A400A5017108A0007208A1008A1154
:10095000172083122608F3002708F4007408F60015
:1009600030307307F5000318F60A75088A11F22073
:100970000A308312A400A5016D08A0006E08A10032
:100980008A11172083122208F1002308F20072084E
:10099000F40030307107F3000318F40A73088A1169
:1009A000F2202A308A11F2200D308A11F2200A300A
:1009B0008A11F2288312EB0014306B02031D132DF1
:1009C0002030F22020308A11F22020308A11F220CB
:1009D00041308A11F22072308A11F2206D308A1172
:1009E000F22020308A11F22070308A11F2206F300C
:1009F0008A11F22073308A11F22069308A11F220B4
:100A000074308A11F22069308A11F2206F308A1115
:100A1000F2206E308A11F22083123408ED0035087E
:100A2000EE008A111E23153083126B028A11031DFA
:100A30004B2D3130F22031308A11F2202E308A11C4
:100A4000F22041308A11F22072308A11F2206D308A
:100A50008A11F22020308A11F22064308A11F220AB
:100A600065308A11F2206C308A11F22061308A11CF
:100A7000F22079308A11F22020308A11F2202030C1
:100A80008A11F22020308A11F22083124D08ED00E5
:100A9000EE018A111E23163083126B028A11031D88
:100AA000832D3130F22032308A11F2202E308A111B
:100AB000F22050308A11F22061308A11F220703019
:100AC0008A11F22065308A11F22072308A11F220E8
:100AD00020308A11F22064308A11F22065308A11A8
:100AE000F2206C308A11F22061308A11F2207930C4
:100AF0008A11F22020308A11F22083124E08ED0074
:100B0000EE018A111E23173083126B028A11031D16
:100B1000BB2D3130F22033308A11F2202E308A1171
:100B2000F22050308A11F22075308A11F2206E3096
:100B30008A11F22063308A11F22068308A11F22083
:100B400020308A11F22064308A11F22065308A1137
:100B5000F2206C308A11F22061308A11F220793053
:100B60008A11F22020308A11F22083124F08ED0002
:100B7000EE018A111E23183083126B028A11031DA5
:100B8000F32D3130F22034308A11F2202E308A11C8
:100B9000F22041308A11F22072308A11F2206D3039
:100BA0008A11F22073308A11F22074308A11F220F7
:100BB00065308A11F22070308A11F22020308A11BB
:100BC000F22066308A11F22061308A11F2206330FF
:100BD0008A11F22074308A11F22083125008ED003D
:100BE000EE018A111E23193083126B028A11031D34
:100BF0002B2E3130F22035308A11F2202E308A111E
:100C0000F22050308A11F22061308A11F2207030C7
:100C10008A11F22065308A11F22072308A11F22096
:100C200073308A11F22074308A11F22065308A11F3
:100C3000F22070308A11F22020308A11F2206630C2
:100C40008A11F22074308A11F22083125108ED00CB
:100C5000EE018A111E231C3083126B028A11031DC0
:100C6000632E3130F22038308A11F2202E308A1172
:100C7000F2204D308A11F22061308A11F220783052
:100C80008A11F22020308A11F22041308A11F2209C
:100C900072308A11F2206D308A11F22020308A11D0
:100CA000F22064308A11F22065308A11F220763009
:100CB0008A11F22020308A11F22083125208ED00AE
:100CC000EE018A111E231D3083126B028A11031D4F
:100CD0008C2E4130F22072308A11F2206D308A1150
:100CE000F22020308A11F22044308A11F22065303F
:100CF0008A11F22076308A11F2202E308A11F220E9
:100D00003A308A11F22020308A11F22083125308DF
:100D1000ED00EE018A111E231E3083126B028A1130
:100D2000031DBF2E4830F22061308A11F2206E3050
:100D30008A11F22073308A11F22020308A11F220B9
:100D400050308A11F2206F308A11F2206E308A11F1
:100D5000F22073308A11F22020308A11F2202330E1
:100D60008312ED00EE018A111E232F308A11F2202A
:100D7000DD308312ED000730EE008A111E2B0800D3
:100D80000130C2208312CD0002308A11C2208312AA
:100D9000CE0003308A11C2208312CF0004308A11A2
:100DA000C2208312D00005308A11C2208312D100E4
:100DB00008308A11C2208312D2001E304D026F10FB
:100DC0008A110319E52E03186F1405304D02EF1038
:100DD0000319EC2E031CEF146F116F1CEF186F1525
:100DE0006F1DF42E0A30CD001E304E02EF11031994
:100DF000FB2E0318EF1505304E026F120319022F58
:100E0000031C6F16EF12EF1D6F1AEF16EF1E0A2F5D
:100E10000A30CE00C8304F020319122F031C122FC4
:100E20000530CF000330500203191A2F031C1A2F6C
:100E30000130D000033051020319222F031C222F4E
:100E40000130D1001E30520203192A2F031C2A2F11
:100E50000530D2000800C0268312EB0131088A1148
:100E600012228312B1007108B00031088A116C207F
:100E700083124D088A1188208312EB0A0A306B0214
:100E80008A11031D2E2F83120618552F31081222A6
:100E90008312B1007108B00031088A116C208312EE
:100EA0004D088A1188208A11432FED013108532201
:100EB0008312B1007108B00031088A116C208312CE
:100EC0004D088A1188208312ED0A32306D028A1192
:100ED000031D562F0130B400B5010618822F3108CA
:100EE00053228312B1007108B00031088A116C20BE
:100EF00083124D088A1188208312B40A0319B50A97
:100F00008A116D2F3408BC003508BD00DF150800BC
:100F100083126910061869140315DF1D922F691CCE
:100F2000932F942F691803110319C02F35083D0220
:100F3000031D9C2F34083C020319A92F0318A92F65
:100F40003D083502D4003C083402D300031CD4030E
:100F5000B12F35083D02D40034083C02D300031CF5
:100F6000D403FE0154087E02031DB82F5308520219
:100F70000319C02F0318C02F1D30DA248A112B2724
:100F80008312DF116918DF1508008312AE152E08D1
:100F900086004F08222183128A11851ED02FCB2F65
:100FA000AE112E088600013022298312851ED92F0A
:100FB000C527831234083602A00035083702200402
:100FC0008A1503193D283708803AA0003508803A71
:100FD00020028A11031DEE2F340836028A150319E8
:100FE0000E28031C0E283508E50006303407E400FF
:100FF0000318E50A3708803AA0006508803A200205
:10100000031D04286408360203190C2803180C2851
:101010008A11DA228A150E288A119422831237083F
:10102000803AA0003508803A20028A15031D1A284C
:101030003408360203193928031839283708E5001F
:1010400006303607E4000318E50A6508803AA00078
:101050003508803A2002031D2F2834086402031942
:101060003728031837288A11A7228A1539288A11A8
:10107000EB228A1188278A11D92F08008312851E36
:1010800043288A11C527831238083A02A00039087C
:101090003B0220048A150319A3283B08803AA000CC
:1010A0003908803A2002031D572838083A020319EC
:1010B0007628031C76283908E50006303807E40056
:1010C0000318E50A3B08803AA0006508803A200230
:1010D000031D6C2864083A02031974280318742845
:1010E0008A110D238A1576288A11C92283123B089A
:1010F000803AA0003908803A20028A15031D822810
:1011000038083A0203194328031843283B08E5002E
:1011100006303A07E4000318E50A6508803AA000A3
:101120003908803A2002031D972838086402031901
:101130009F2803189F288A11B8228A1543288A11EC
:10114000FC228A154328B801B90108001E308A1113
:10115000DA2483128A15061CAE28A928851EB22817
:101160008A11C5278A112B278312B601B7018A116C
:10117000D52783122D122D08850001308A11882071
:101180008A11FC208312AF005F1320185F178A15A5
:101190005F1FB92824302F02031DD028B301DF14AC
:1011A00023302F02031DD628B3015F15E010DF1C8A
:1011B0005F19E014E01CE4284230330784008313F5
:1011C00030302F028000B30A0A3033020319B928E5
:1011D000031CB9282D162D0885005F1DDA2A5F1122
:1011E000B3014408A000A101E830A2000330A3002D
:1011F0008A11042083122408D5002508D60045084A
:10120000A000A1016430A200A3018A11042083126E
:101210002408D7002508D80058085607DA005708D0
:101220005507D9000318DA0A4608A000A1010A30C0
:10123000A200A3018A11042083122408DB002508E0
:10124000DC005C085A07DE005B085907DD00031864
:10125000DE0A5E08BF0047085D07BE000318BF0A2C
:101260004908A000A101E830A2000330A3008A11C0
:10127000042083122408D5002508D6004A08A000BF
:10128000A1016430A200A3018A1104208312240862
:10129000D7002508D80058085607DA005708550720
:1012A000D9000318DA0A4B08A000A1010A30A200F5
:1012B000A3018A11042083122408DB002508DC0026
:1012C0005C085A07DE005B085907DD000318DE0AD8
:1012D0005E08C1004C085D07C0000318C10A42083F
:1012E000E400E5013E08E9003F08EA004008ED009F
:1012F0004108EE008A11AB23013083123E02A000A8
:1013000000303F0220048A15031DA1294008A000D7
:101310004108A1005008A200A3018A1104208312F1
:101320002408C0002508C10041083507B70040085F
:101330003407B6000318B70A8A11D52714308A116A
:10134000DA24023083123E02A00000303F02200463
:101350008A15031DD5294008A0004108A1005008A6
:10136000A200A3018A11042083122408C0002508CA
:10137000C100350841028A15031DC0293408400206
:101380000319CD290318CD2941083502B7004008BB
:101390003402B600031CB703D0290130B600B701F0
:1013A0008A11D52714308A11DA24033083123E02C1
:1013B000A00000303F0220048A15031DF3294008D5
:1013C000A0004108A1005108A200A3018A11042035
:1013D00083122408C0002508C1004008BA00410853
:1013E000BB008A153E20043083123E02A00000306C
:1013F0003F0220048A15031D052A0130B600B701FB
:101400008A11D52714308A11DA24053083123E025E
:10141000A00000303F0220048A15031D182A3C0852
:10142000B6003D08B7008A11D52714308A11DA2496
:10143000063083123E02A00000303F0220048A15CD
:10144000031D242A8A11C527073083123E02A000FB
:1014500000303F0220048A15031D362A4008B800D8
:101460004108B9000130BA00BB013E200B308312A5
:101470003E02A00000303F0220048A15031D4A2AC4
:101480004008E60001308A11CD208A11C0261530AF
:101490008A11DA240C3083123E02A00000303F0291
:1014A00020048A15031D5E2A4008E60002308A11D6
:1014B000CD208A11C02616308A11DA240D3083120D
:1014C0003E02A00000303F0220048A15031D722A4C
:1014D0004008E60003308A11CD208A11C02617305B
:1014E0008A11DA240E3083123E02A00000303F023F
:1014F00020048A15031D862A4008E60004308A115C
:10150000CD208A11C02618308A11DA240F308312B8
:101510003E02A00000303F0220048A15031D9A2AD3
:101520004008E60005308A11CD208A11C026193006
:101530008A11DA24123083123E02A00000303F02EA
:1015400020048A15031DAE2A4008E60008308A11DF
:10155000CD208A11C0261C308A11DA241330831260
:101560003E02A00000303F0220048A15031DBE2A5F
:101570008A112B2714308312BE00BF0114303E02A3
:10158000A00000303F0220048A15031DD82A8A11CA
:10159000C0268312E3013E088A11DA248312BE0AB0
:1015A0000319BF0AE30A0B3063028A15031DCB2A15
:1015B000BE01BF01DF1CB928DF10B3014408A00041
:1015C000A101E830A2000330A3008A110420831295
:1015D0002408D5002508D6004508A000A1016430E4
:1015E000A200A3018A11042083122408D700250831
:1015F000D80058085607DA0057085507D9000318CD
:10160000DA0A4608A000A1010A30A200A3018A114B
:10161000042083122408DB002508DC005C085A073C
:10162000DE005B085907DD000318DE0A5E08B7001C
:1016300047085D07B6000318B70A3608A000370848
:10164000A1005008A200A3018A11042083122408DB
:10165000B6002508B7004908A000A101E830A200A3
:101660000330A3008A11042083122408D500250822
:10167000D6004A08A000A1016430A200A3018A118B
:10168000042083122408D7002508D80058085607DC
:10169000DA0057085507D9000318DA0A4B08A000EA
:1016A000A1010A30A200A3018A1104208312240898
:1016B000DB002508DC005C085A07DE005B085907E0
:1016C000DD000318DE0A5E08BB004C085D07BA00A7
:1016D0000318BB0A3A08A0003B08A1005108A20069
:1016E000A3018A11042083122408BA002508BB0034
:1016F0004208E400E5013608E9003708EA003A0844
:10170000ED003B08EE008A11AB238A153E208A11BA
:0A171000D5278A11C5278A15B928CC
:02400E00023D71
:00000001FF
